:020000040000FA
:06000000C5EF01F0120043
:06002A000100C603000006
:08003000600000001000000058
:08003800816A936A806A9268F4
:1000400000017C6B7E6B806B0B0EE66E040EE66E21
:10005000910EE66E37EC01F0E552E552E5520001F3
:100060007E51080DF350E66E8AEC01F0E552240E45
:10007000E66ED1EC01F0E552E1EC01F0DCEC01F0D0
:10008000000901E0FBD76BEC01F0F3CF7AF0F4CF7D
:100090007BF000017D6B7C51E76E7D19E8AE02D0EC
:1000A000E73402D0E7507D5D10E20A0E0B6E0C6A59
:1000B0007AC006F07BC007F011EC01F006C07AF0C0
:1000C00007C07BF000017D2BE6D77AC010F07BC023
:1000D00011F00A0E0B6E0C6A10C006F011C007F08A
:1000E00011EC01F002C010F003C011F010C07FF05D
:1000F000040E00017C25106E010E105204E0E8464B
:10010000FE0B1006FCE100017F11816E030EE76E0D
:100110007C19E8AE02D0E73402D0E7507C5D02E201
:100120007C2B01D07C6B80A803D0010E806F0ED099
:1001300080510AE07E29106E10C007F0040E0C6E8C
:10014000F7EC00F003C07EF00001806B88D712004E
:100150002A0EF66E000EF76E000EF86E0001090012
:10016000F550756F0900F550766F03E1756701D0A2
:100170003DD00900F550706F0900F550716F09000E
:10018000F550726F09000900F550E96E0900F5504D
:10019000EA6E090009000900F550736F0900F55077
:1001A000746F09000900F6CF77F0F7CF78F0F8CF39
:1001B00079F070C0F6FF71C0F7FF72C0F8FF000160
:1001C000735302E1745307E00900F550EE6E7307B4
:1001D000F8E27407F9D777C0F6FF78C0F7FF79C067
:0E01E000F8FF00017507000E765BBFD7120016
:0201EE000E6A97
:1001F0000CAEFDEF00F00C6C0E1E07AE02EF01F02E
:10020000076C0E1EB7EC01F007BE0CEF01F00EAE4E
:10021000000C076C036C000C0EBE09EF01F00F8898
:10022000FF0C0E6A0CAE1AEF01F00B6C0C1EE86AA4
:100230000C220E1E07AE22EF01F0066C071EE86AC4
:1002400007220E1EA1EC01F007BE32EF01F00EAE48
:10025000000C066C071EE86A0722026C031EE86A9F
:0E0260000322000C0EBE29EF01F00F88FF0CE8
:02026E00D9CFE6
:10027000E6FFDACFE6FFE1CFD9FFE2CFDAFFC26ACD
:10028000C16AC06AFC0EDB407F0B3C0BC26EFB0EEA
:10029000DB50C16EFC0EDB38F00B300BC112FD0ED3
:1002A000DB50800BC06EFD0EDB380F0B070BC0124E
:1002B000FD0EDB50040DF350380BC012FC0EDBAE0C
:1002C00003D09E9C9D8CF28CC280E552E5CFDAFF74
:0602D000E7CFD9FF120088
:0A02D600D9CFE6FFDACFE6FFE1CF53
:1002E000D9FFE2CFDAFFE652E652C350DF6E010ECD
:1002F000C4CFDBFFDECF10F0DDCF11F010C0F3FF75
:1003000011C0F4FFE552E552E552E5CFDAFFE7CF41
:04031000D9FF1200FF
:0C031400D9CFE6FFDACFE6FFE1CFD9FF3A
:10032000E2CFDAFFC30EC214106EFD0EDB407F0B6E
:100330003C0B1010C26EE552E5CFDAFFE7CFD9FFD4
:020340001200A9
:0E034200036A026A100EE76ED8900636073680
:10035000023603360B50025C0C50035805E30B5079
:0E036000025E0C50035A062AE72EF0D7120058
:02036E00036A20
:10037000080EE76ED890073603360C50035C02E394
:0A038000036E072AE72EF7D71200DC
:06038A0013EE00F023EE6B
:1003900000F0F86A0F9CA8EC00F01CEC00F0FDD710
:0203A000120049
:0E03A200FF0EE350E84E1200000000D000D025
:0803B00000D0E82EFAD712007C
:0803B800C250020B01E0010E2E
:0203C000120029
:0403C200C2821200E1
:0A03C6003F065B4F666D7D077F6FF9
:0603D000777C395E7971B3
:020000040030CA
:0E000000100F1F1E008181000FC00FE00F4087
:00000001FF
